:100000000C94EB010C9408020C9408020C94080266
:100010000C9408020C9408020C9408020C94080238
:100020000C9408020C94E9120C9408020C943014FD
:100030000C9408020C9408020C9408020C94080218
:100040000C9408020C9408020C949C100C9455100B
:100050000C9408020C9408020C9408020C940802F8
:100060000C9408020C940802084AD73B3BCE016E60
:1000700084BCBFFDC12F3D6C74319ABD56833DDAFF
:100080003D00C77F11BED9E4BB4C3E916BAAAABE0E
:10009000000000803F05A84CCDB2D44EB93836A937
:1000A000020C50B9918688083CA6AAAA2ABE000074
:1000B00000803F0D0A00496E76616C696420636FB1
:1000C0006D6D616E640D0A004D6F64616C20677226
:1000D0006F75702076696F6C6174696F6E0D0A00C0
:1000E000466C6F6174696E6720706F696E7420650D
:1000F00072726F720D0A00556E737570706F727444
:1001000065642073746174656D656E740D0A0045D5
:100110007870656374656420636F6D6D616E6420D3
:100120006C65747465720D0A00426164206E756DB1
:1001300062657220666F726D61740D0A006572727D
:100140006F723A20006F6B0D0A000D0A27242720DA
:10015000746F2064756D702063757272656E7420A3
:1001600073657474696E67730D0A000D0A477262D5
:100170006C20302E3861005761726E696E673A20CC
:100180004661696C656420746F2072656164204506
:100190004550524F4D2073657474696E67732E20FD
:1001A0005573696E672064656661756C74732E0D96
:1001B0000A0053746F726564206E657720736574EE
:1001C00074696E670D0A00556E6B6E6F776E2070E6
:1001D0006172616D657465720D0A005374657020FB
:1001E00070756C7365206D757374206265203E3D7B
:1001F0002033206D6963726F7365636F6E64730D76
:100200000A0053746570732F6D6D206D75737420C3
:100210006265203E20302E300D0A000D0A2724781A
:100220003D76616C75652720746F2073657420704E
:100230006172616D65746572206F72206A75737486
:100240002027242720746F2064756D7020637572D9
:1002500072656E742073657474696E67730D0A003D
:100260002028636F726E6572696E67206A756E63AF
:1002700074696F6E20646576696174696F6E206958
:100280006E206D6D29002028616363656C65726165
:1002900074696F6E20696E206D6D2F7365635E32B9
:1002A000290D0A2439203D2000290D0A2438203D3B
:1002B000200020287374657020706F727420696E3E
:1002C00076657274206D61736B2E2062696E617247
:1002D00079203D200020286D6D2F617263207365A9
:1002E000676D656E74290D0A2437203D2000202893
:1002F0006D6D2F6D696E2064656661756C74207319
:1003000065656B2072617465290D0A2436203D20D5
:100310000020286D6D2F6D696E2064656661756CB7
:100320007420666565642072617465290D0A243540
:10033000203D200020286D6963726F7365636F6EC6
:10034000647320737465702070756C7365290D0A71
:100350002434203D2000202873746570732F6D6D48
:10036000207A290D0A2433203D200020287374654B
:1003700070732F6D6D2079290D0A2432203D2000E5
:10038000202873746570732F6D6D2078290D0A24F1
:1003900031203D20002430203D2000494E46494E6A
:1003A0004954594E414ECDCCCC3D0AD7233C17B7CA
:1003B000D13877CC2B329595E6241FB14F0A000037
:1003C00020410000C84200401C4620BCBE4CCA1B55
:1003D0000E5AAEC59D7411241FBECFEFD8E0DEBF0C
:1003E000CDBF11E0A0E0B1E0E4EDF4E502C005907E
:1003F0000D92A631B107D9F716E0A6E1B1E001C030
:100400001D92AD3EB107E1F70E9482030C94682A69
:100410000C940000A0E0B0E0E0E1F2E00C94372A98
:10042000EC015B016115710519F0FB01918380837B
:10043000F9908F2D90E00E94262A892BC9F7FDE2C2
:10044000FF1621F4F990EE24E39405C02BE2F21696
:1004500009F4F990EE248E0101501040C8016BE9B7
:1004600073E043E050E00E946A03892B01F58E019E
:100470000E5F1F4FC8016EE973E045E050E00E9437
:100480006A03892B19F48E01095F1F4FA114B1046F
:1004900019F0F50111830083E0FC04C070E090E0E6
:1004A00080E814C070E090E080E86FEF08C1C801F8
:1004B00063EA73E043E050E00E946A03892B69F429
:1004C000A114B10429F470E090E080EC6FE7F7C06C
:1004D0002296F501D183C083F6CF8824992440E089
:1004E00050E060E070E0EF2DE053EA30A0F5F2E07C
:1004F000EF2A8E2D90E09C0128703070E2FE06C03D
:10050000232B79F50894811C911C2BC0232B19F007
:10051000089481089108DB01CA0112E0880F991F35
:10052000AA1FBB1F1A95D1F7480F591F6A1F7B1FBF
:10053000440F551F661F771F4E0F511D611D711D02
:10054000483929E9520729E9620729E1720748F089
:1005500084E0E82A06C0EE3F31F4E3FC39C098E0BD
:10056000E92AF990C0CFE53311F0E53189F52991F9
:100570002D3219F4E0E1EE2A05C02B3219F081E0AA
:1005800090E003C0299182E090E0E22FE053EA304E
:1005900018F0C81BD90B1CC020E030E0FCE020386C
:1005A0003F075CF4C901880F991F880F991F280F16
:1005B000391F220F331F2E0F311DE991E053EA300E
:1005C00068F3E4FE03C0309521953F4F820E931EE1
:1005D000CE2CDD24E1FE07C0A114B10421F0219747
:1005E000F501D183C083CB01BA010E948D267B0126
:1005F0008C01F3E0CF22DD2423E0C216D10421F4E4
:1006000017FB109517F9109557016801C801B7013C
:1006100020E030E040E050E00E94ED25882309F41E
:100620004AC097FE0DC02AEBE22E23E0F22E9094F2
:10063000819491089394C0E2D0E000E010E012C0F1
:1006400092EDE92E93E0F92EF6CFF7012591359141
:1006500045915491C601B5010E94CD285B016C0102
:100660008C1A9D0A8C169D0684F7D595C7950F5F49
:100670001F4F0630110529F08CEF9FEFE80EF91E91
:10068000F1CFC501D6017C018D018C2D880F8D2DF8
:10069000881F8F3F51F0C601B50120E030E040E0F7
:1006A00050E00E94ED25882331F482E290E090939F
:1006B000EC068093EB067E2D9F2D802F612F272F38
:1006C000392F482F562FB901CA01CDB7DEB7ECE05C
:1006D0000C94532AFB01DC014150504088F08D916D
:1006E00081341CF08B350CF4805E659161341CF014
:1006F0006B350CF4605E861B611171F3990B0895E4
:10070000881BFCCF6F927F928F929F92AF92BF9285
:10071000CF92DF92EF92FF920F931F93DF93CF93CD
:10072000CDB7DEB768970FB6F894DEBF0FBECDBF6A
:1007300060E875E280E090E00E9407100E940013DC
:100740007894EEEDF5E08AE2DF011D928A95E9F7F3
:1007500081E08093DE055E010894A11CB11C9DE040
:10076000C92ED12CCC0EDD1E4F018AE2682E7724D3
:1007700073948091DE05882309F453C0D501E1EE1E
:10078000F5E08CE001900D928150E1F7D601EEEE9C
:10079000F5E08CE001900D928150E1F7F401862D97
:1007A00011928A95E9F70E9497100E944B1A0E94B5
:1007B000F7100E94CF220E9441080E94E40F0E947D
:1007C00031230E941C14A1EEB5E0F5018CE00190EC
:1007D0000D928150E1F7AEEEB5E0F6018CE00190AC
:1007E0000D928150E1F769817A818B819C812D8105
:1007F0003E814F815885E984FA840B851C850E94CF
:10080000EE0769817A818B819C812D813E814F81A8
:100810005885E984FA840B851C850E94401B7092E0
:10082000E0050E9451120E948812A3CFEF92FF921E
:100830000F931F930E949F2360E070E080E090E0A0
:1008400020E030E040E050E0EE24FF2487010E94E9
:10085000401B1F910F91FF90EF900895EF92FF9230
:100860000F931F93CF93DF937B018C0120E030E047
:1008700040EA51E40E94CD280E94CA260E946126C7
:10088000EB010E94B222C801B70120E030E04AE744
:1008900054E40E94CD287B018C0182E390E0C89F44
:1008A000B001C99F700DD89F700D112480E090E0B9
:1008B0000E948D269B01AC01C801B7010E9413253F
:1008C0000E94CA260E946126DC01CB010E94E3221D
:1008D00000E911E00EC00E9451128091DE058823CC
:1008E00051F484EF91E0F8013197F1F70197D9F7CE
:1008F0002197209781F7DF91CF911F910F91FF9062
:10090000EF9008954F925F926F927F928F92AF9285
:10091000BF92CF92DF92EF92FF920F931F93DF93DC
:10092000CF9300D000D0CDB7DEB72B013C01298397
:100930003A834B835C830E9451128091DE058823A9
:1009400091F40E94361B8823B1F7C301B2012981BB
:100950003A814B815C810E94C71E8091E00588230B
:1009600011F00E94AC130F900F900F900F90CF9149
:10097000DF911F910F91FF90EF90DF90CF90BF908C
:10098000AF908F907F906F905F904F9008952F92CF
:100990003F924F925F926F927F928F929F92AF920F
:1009A000BF92CF92DF92EF92FF920F931F93DF934C
:1009B000CF93CDB7DEB7CE54D0400FB6F894DEBF9C
:1009C0000FBECDBF3C017EAF6DAF21965FAF4EAF86
:1009D000219722962FAF229723960FAF2397249625
:1009E000EFAE24972896ACAEBDAECEAEDFAE289764
:1009F00029968FAE2997E22EFF24EE0CFF1CEE0CF9
:100A0000FF1C4E0D5F1D5CAF4BAFDA012D903D908A
:100A10004D905C90FC01EE0DFF1DC201B1012081E3
:100A20003181428153810E94142569AB7AAB8BAB33
:100A30009CAB10E0000F111F000F111F2196EEADAF
:100A4000FFAD2197E00FF11FFAAFE9AFA080B180B1
:100A5000C280D380F301E00FF11FC601B5012081F0
:100A60003181428153810E9414256DA77EA78FA7F3
:100A700098AB24962FAD2497E22FF0E0EE0FFF1FE6
:100A8000EE0FFF1F6E0E7F1ED3018D919D910D9075
:100A9000BC91A02D8DAB9EABAFABB8AF2DAD3EAD35
:100AA000E20FF31F60817181828193812DA93EA99C
:100AB0004FA958AD0E94132569A77AA78BA79CA7B9
:100AC000D201C101B0588DA39EA3AFA3B8A7A601C0
:100AD0009501505829A33AA34BA35CA34DAD5EAD3D
:100AE000E40EF51ED7016D917D918D919C9129A900
:100AF0003AA94BA95CA90E9413253B014C01EDAD1D
:100B0000FEAD0E0F1F1FD8016D917D918D919C91AF
:100B10002DA53EA54FA558A90E9413255B016C0188
:100B20006DA17EA18FA198A5A60195010E94CD2857
:100B30007B018C0169A17AA18BA19CA1A4019301E5
:100B40000E94CD289B01AC01C801B7010E9413256A
:100B50001B012C016DA17EA18FA198A5A401930179
:100B60000E94CD287B018C0169A17AA18BA19CA157
:100B7000A60195010E94CD289B01AC01C801B701D7
:100B80000E9414259B01AC01C201B1010E9487257E
:100B90005B016C0120E030E040E050E00E94ED2578
:100BA000882354F4C601B5012BED3FE049EC50E435
:100BB0000E9414255B016C01A8968FADA89788232D
:100BC00051F0C601B5012BED3FE049EC50E40E9425
:100BD00013255B016C01C601B501A7962CAD3DAD97
:100BE0004EAD5FADA7970E94CD2829A53AA54BA58C
:100BF0005CA50E9408287B018C0120E030E040E0E9
:100C000050E00E94ED25882309F4CEC1C801B70148
:100C10002091DF063091E0064091E1065091E20616
:100C20000E94F4250E94CA260E94612678A36F8F35
:100C30002996BFAD2997BB23A1F080E090E00E94E8
:100C40008D269B01AC0128966CAD7DAD8EAD9FAD20
:100C500028970E94CD2828966CAF7DAF8EAF9FAFAE
:100C600028972F8D38A1B90180E090E00E948D2651
:100C70007B018C01C601B501A80197010E94F425F2
:100C80006B8F7C8F8D8F9E8F69A57AA58BA59CA578
:100C9000A80197010E94F4256F8B788F898F9A8F16
:100CA0006B8D7C8D8D8D9E8D20E030E040E05FEB84
:100CB0000E94CD282B8D3C8D4D8D5E8D0E94CD28C0
:100CC00020E030E040E85FE30E9414256B8B7C8BD2
:100CD0008D8B9E8B24963FAD2497E32FF0E0EE0F93
:100CE000FF1FEE0FFF1FCE010196E80FF91F2DA980
:100CF0003EA94FA958AD208331834283538341E0FD
:100D000050E05E874D8766242296BFAD2297AB2FB9
:100D1000B0E0AA0FBB1FAA0FBB1FA80FB91F2B96CD
:100D2000BFAFAEAF2B9723963FAD2397232F30E075
:100D3000220F331F220F331F280F391F2D963FAF6D
:100D40002EAF2D972F96FFAFEEAF2F9707C148E13B
:100D500046150CF446C06DA17EA18FA198A52B8DE0
:100D60003C8D4D8D5E8D0E94CD287B018C0169A14B
:100D70007AA18BA19CA12B893C894D895E890E9417
:100D8000CD289B01AC01C801B7010E9414257B014D
:100D90008C016DA17EA18FA198A52B893C894D89DD
:100DA0005E890E94CD285B016C0169A17AA18BA1AB
:100DB0009CA12B8D3C8D4D8D5E8D0E94CD289B017D
:100DC000AC01C601B5010E9413256DA37EA38FA3BC
:100DD00098A76394C701D80189A39AA3ABA3BCA326
:100DE00061C0AD85BE85BD0180E090E00E948D268A
:100DF0002B8D3C8D4D8D5E8D0E94CD287B018C010D
:100E0000C8010E94F1256F87788B898B9A8BB70177
:100E1000C8010E9450293B014C01EBADFCADE080C4
:100E2000F1800281138117FB109517F91095A9AD78
:100E3000BAAD2D903D904D905C90C801B7012F85C3
:100E4000388949895A890E94CD285B016C01C20109
:100E5000B101A40193010E94CD289B01AC01C60100
:100E6000B5010E9414256DA37EA38FA398A7C80186
:100E7000B701A40193010E94CD287B018C01C2011E
:100E8000B1012F85388949895A890E94CD289B0153
:100E9000AC01C801B7010E94132569A37AA38BA3F3
:100EA0009CA3662469A97AA98BA99CA92DA13EA11E
:100EB0004FA158A50E9414252B96EEADFFAD2B97A0
:100EC00060837183828393836DA57EA58FA598A986
:100ED00029A13AA14BA15CA10E9414252D96AEAD8B
:100EE000BFAD2D976D937D938D939C9313972F9604
:100EF000EEADFFAD2F9760817181828193812F8943
:100F0000388D498D5A8D0E9414252F96AEADBFADF8
:100F10002F976D937D938D939C93139769817A811D
:100F20008B819C812D813E814F815885E984FA8493
:100F30000B851C852896ACACBDACCEACDFAC28973D
:100F400029968FAC29970E9482048091DE05882320
:100F500059F5ED85FE853196FE87ED872D853E8519
:100F60004F8D58A12417350708F4F1CEADADBEADB5
:100F70006D917D918D919C91139714962D913D913A
:100F80004D915C9117971896ED90FD900D911C91E5
:100F90001B972896ACACBDACCEACDFAC289729969D
:100FA0008FAC29970E948204C25BDF4F0FB6F89482
:100FB000DEBF0FBECDBFCF91DF911F910F91FF908C
:100FC000EF90DF90CF90BF90AF909F908F907F90E9
:100FD0006F905F904F903F902F900895AF92BF9287
:100FE000CF92DF92EF92FF920F931F9359016A0104
:100FF0000E948F262091C8063091C9064091CA06EA
:101000005091CB060E94F425609325017093260130
:101010008093270190932801C601B5010E948F2675
:101020002091CC063091CD064091CE065091CF064E
:101030000E94F4256093290170932A0180932B016B
:1010400090932C01C801B7010E948F262091D006F1
:101050003091D1064091D2065091D3060E94F425DA
:1010600060932D0170932E0180932F019093300196
:101070001F910F91FF90EF90DF90CF90BF90AF90B6
:10108000089581E2E6E1F1E0DF011D928A95E9F73A
:101090008091D6069091D706A091D806B091D90636
:1010A00080931D0190931E01A0931F01B093200116
:1010B0001092340191E09093350182E080933601E3
:1010C00090931A0108952F923F924F925F926F92E0
:1010D0007F928F929F92AF92BF92CF92DF92EF92C8
:1010E000FF920F931F93DF93CF93CDB7DEB7A897EF
:1010F0000FB6F894DEBF0FBECDBF3C0119828CE065
:10110000FE013696DF01482F1D924A95E9F7FE0150
:101110007296DF011D928A95E9F710921601442418
:1011200055241CA21BA262E0262E312C2C0E3D1E43
:1011300001E053E0A52E42E0B42E31E0832E912C45
:101140006BC12E313105C9F12F313105D4F4243171
:10115000310584F421313105A4F52430310569F1DC
:10116000253031051CF437FF2AC025C02A3031054F
:1011700011F523C02631310554F12C313105D9F454
:101180001CC02C3531058CF42A353105E4F42C33A0
:1011900031053CF426333105E4F42533310559F4A7
:1011A0000CC02035310539F40AC02C35310529F041
:1011B0002F35310554F010E00DC011E00BC012E0E6
:1011C00009C013E007C014E005C016E003C017E033
:1011D00001C019E02531310509F495C026313105EA
:1011E000A4F52430310509F467C025303105A4F495
:1011F0002130310509F466C02230310524F4232B57
:1012000009F45DC0F4C02230310509F45EC023301A
:10121000310509F0ECC05CC02231310509F462C02F
:10122000233131054CF42A30310509F443C0213112
:10123000310509F0DCC04FC02331310509F459C034
:101240002431310509F0D3C05BC02035310509F4E4
:101250006AC021353105ACF42533310509F459C094
:10126000263331054CF42C31310509F44FC02E31B1
:10127000310509F0BCC04AC02C3331050CF0B7C0B1
:101280004BC02C35310509F458C02D3531054CF4CF
:101290002A35310509F44BC02B35310509F0A7C0BB
:1012A00049C02D35310509F462C02E35310509F0EC
:1012B0009EC060C0B2E059C0E1E0EBA39AC01092BA
:1012C000170197C00093170194C0B092170191C005
:1012D000A09217018EC01092340100933501B09294
:1012E000360187C010923401B09235010093360167
:1012F00080C000933401B09235011092360179C05C
:101300000093190176C01092190173C0F3E0FBA39A
:1013100070C041E04CA36DC02633310509F067C0B1
:101320001092ED0566C054E05093170162C000931F
:101330001A015FC010921A015CC0C701B60120E01B
:1013400030E040E251E40E94CD280E94A7290E948B
:101350005C2683E06839780739F06959734009F0F1
:1013600046C0A5E0ABA345C0B4E0BBA342C0009318
:1013700018013FC0109218013CC02630310534F4EA
:101380002330310554F4772334F403C02E31310572
:1013900011F010E003C015E001C018E02330310562
:1013A000E1F0243031054CF42130310581F0223058
:1013B000310584F4232B59F01AC025303105A1F0F2
:1013C000253031056CF02E31310589F403C00093CE
:1013D0001B010FC0B0921B010CC000931C0109C07F
:1013E000EFEFE0931C0105C010921C0102C0A09217
:1013F0001601112389F0940102C0220F331F1A95A0
:10140000E2F7C90184219521892B21F0F5E0F093C1
:10141000160102C0422A532A9981F301E90FF11DF6
:1014200010811123A9F0812F81548A3110F082E0BC
:101430000DC09F5F9983C301BE016F5F7F4FA10104
:101440000E94F622892B09F085C581E08093160160
:1014500080911601882309F064C5198299241DA280
:101460001EA240E84FA35FEB58A70F2EF0E0AF2E6F
:10147000F0E0BF2EF0E0CF2EF0E0DF2EF02DAF8EAB
:10148000B8A2C9A2DAA21E8E1E010894211C311C2A
:1014900026E0822E11C1EA80FB800C811D81C801EB
:1014A000B70120E030E040E050E00E94ED25181642
:1014B00014F08092160180911801882381F08091A8
:1014C0001901882309F4F2C0C801B70123E333E30B
:1014D0004BEC51E40E94CD287B018C01E7C0809148
:1014E0001901882351F0C801B70123E333E34BEC22
:1014F00051E40E94CD287B018C01E0921D01F09205
:101500001E0100931F0110932001CAC02A813B8154
:101510004C815D8180911901882351F0CA01B90184
:1015200023E333E34BEC51E40E94CD289B01AC0153
:10153000E12FFF27E7FDF095E954F040EE0FFF1F84
:10154000EE0FFF1FE20DF31D218B328B438B548B6B
:10155000A7C06A817B818C819D810E94A7290E94FE
:1015600061266E8F9DC0AA80BB80CC80DD8098C034
:101570006A817B818C819D816F8F78A389A39AA3D7
:1015800080911901882309F48BC06F8D78A189A1FE
:101590009AA123E333E34BEC51E40E94CD286F8FF3
:1015A00078A389A39AA37CC0EA80FB800C811D816B
:1015B000C801B70120E030E040E050E00E94ED2596
:1015C000882314F480921601C801B7010E945C269A
:1015D000709333016093320163C0EA80FB800C8119
:1015E0001D81C801B70120E030E040E050E00E94DA
:1015F000ED25882314F480921601C801B7010E94DA
:10160000A7290E946126609331014AC02A813B814B
:101610004C815D8180911901882351F0CA01B90183
:1016200023E333E34BEC51E40E94CD289B01AC0152
:101630002E833F834887598771E0972A31C02A81DA
:101640003B814C815D8180911901882351F0CA0151
:10165000B90123E333E34BEC51E40E94CD289B0115
:10166000AC012A873B874C875D8782E0982A18C0A7
:101670002A813B814C815D8180911901882351F041
:10168000CA01B90123E333E34BEC51E40E94CD28B6
:101690009B01AC012E873F87488B598B94E0992A98
:1016A0008DA19EA1AFA1B8A57C018D01D801C70174
:1016B000EDA29EA3AFA3B8A79981F301E90FF11D95
:1016C00010811123A9F0812F81548A3110F082E01A
:1016D0000DC09F5F9983C301B101AE014E5F5F4FA3
:1016E0000E94F622892B09F047C481E080931601FD
:1016F00080911601882309F014C480911C01409147
:10170000320150913301662757FD6095762F992756
:1017100087FD90950E94EC0FABA1A33009F457C050
:10172000A43030F4A13061F0A23009F046C118C0F5
:10173000BBA1B43009F4E2C0B53009F03EC134C1F8
:10174000C601B50120E030E040E050E00E94ED2508
:1017500088230CF4D5C0C601B5010E942E042DC10A
:10176000EE8DE23049F4C601B5010E94A7290E941E
:101770005C266130710521F083E0809316011CC165
:10178000992009F4BDC0AE014A5F5F4FEEEEF5E06F
:1017900020E030E0692D70E0CB01022E02C095956B
:1017A00087950A94E2F780FF09C0DA01ED90FD9079
:1017B0000D911C91E082F182028313832F5F3F4FD2
:1017C0004C5F5F4F34962330310531F7F5C09920D7
:1017D00009F48AC08E010A5F1F4F85E2C82E81E09E
:1017E000D82EBAEFAB2EB5E0BB2EEE24FF24892C09
:1017F0009924C4010E2C02C0959587950A94E2F7AE
:1018000080FF41C080911A01882351F18091ED053C
:1018100090E0FC01EE0FFF1FE80FF91FEE0DFF1D1A
:10182000EE0FFF1FEE0FFF1FE251FA4F6081718133
:1018300082819381F50120813181428153810E940F
:1018400014259B01AC01D8016D917D918D919C91E6
:101850000E941425F80160837183828393831DC0E5
:10186000D8016D917D918D919C91F60120813181FE
:10187000428153810E941425D8016D937D938D93ED
:101880009C9313970AC0F60180819181A281B38154
:10189000F80180839183A283B3830894E11CF11C37
:1018A0000C5F1F4F44E050E0C40ED51EA40EB51EC1
:1018B00053E0E516F10409F09CCF6E817F818885A5
:1018C00099852A853B854C855D85EE84FF84088952
:1018D0001989A090DA06B090DB06C090DC06D090A3
:1018E000DD0688240E9482040E9416048CE0E5E252
:1018F000F1E0DF011D928A95E9F75EC0992021F49D
:1019000086E08093160159C065E2A62E61E0B62EEE
:1019100056E0C52ED12CCC0EDD1E4AEFE42E45E05C
:10192000F42E00E010E0892C9924C401002E02C09E
:10193000959587950A94E2F780FF28C08091ED0580
:1019400090E0FC01EE0FFF1FE80FF91FE00FF11F01
:10195000EE0FFF1FEE0FFF1FE251FA4FD5016D9101
:101960007D918D919C9120813181428153810E9492
:101970001325F60120813181428153810E94132574
:10198000D7016D937D938D939C9313970F5F1F4F9A
:10199000E4E0F0E0AE0EBF1ECE0EDF1EEE0EFF1E28
:1019A0000330110511F608C08CE0EAEFF5E0DF0125
:1019B0001D928A95E9F701C0992442FC03C0992041
:1019C00009F4A3C280911801882399F06DA17EA12A
:1019D0008FA198A520E030E040E050E00E94ED2586
:1019E00088233CF480911701843019F086E08093BD
:1019F0001601BCA1BB2339F080911701823018F089
:101A000086E08093160180911601882309F089C22F
:101A10008E010A5F1F4F9AEFA92E95E0B92E85E23D
:101A2000C82E81E0D82EEE24FF24692C7724C30130
:101A30000E2C02C0959587950A94E2F780FF45C069
:101A4000ECA1EE2309F04BC080911A01882359F1D3
:101A50008091ED0590E0FC01EE0FFF1FE80FF91FEC
:101A6000EE0DFF1DEE0FFF1FEE0FFF1FE251FA4FAD
:101A70006081718182819381D5012D913D914D913C
:101A80005C910E9414259B01AC01F8016081718179
:101A9000828193810E941425D8016D937D938D934B
:101AA0009C9313971CC0F80160817181828193819E
:101AB000D6012D913D914D915C910E941425F80124
:101AC00060837183828393830AC0F6018081918150
:101AD000A281B381F80180839183A283B3830894A8
:101AE000E11CF11C0C5F1F4F44E050E0A40EB51E3A
:101AF000C40ED51E53E0E516F10409F098CF80918D
:101B00001701843048F4823008F04CC0882359F023
:101B1000813009F0EDC120C0843009F0E9C199207D
:101B200009F4E6C18BC0992009F488C06E817F81D9
:101B3000888599852A853B854C855D85EE84FF8463
:101B400008891989A090DA06B090DB06C090DC06FF
:101B5000D090DD06882423C0992009F46FC06E81DF
:101B60007F81888599852A853B854C855D85EE84B6
:101B7000FF840889198980901801882061F4A09158
:101B80001D01ADA3B0911E01BEA3E0911F01EFA303
:101B9000F0912001F8A7ADA0BEA0CFA0D8A40E94CC
:101BA0008204A6C181E090E00090360102C0880F57
:101BB000991F0A94E2F78095982209F43FC06F8D2F
:101BC00078A189A19AA120E030E040E050E00E9495
:101BD000ED25882309F043C0E0913401F0E0EE0FD9
:101BE000FF1FEE0FFF1F8E010F5F1F4FE00FF11F52
:101BF000C188D288E388F488C701B60120E030E0CC
:101C000040E050E00E94ED258823E1F48091350109
:101C100090E0880F991F880F991F080F191FD8018E
:101C200051966D917D918D919C91549720E030E07B
:101C300040E050E00E94ED25882321F486E0809367
:101C4000160156C16F8D78A189A19AA120E030E0DC
:101C500040E050E00E94ED25882309F4F2C0E091B5
:101C60003401F0E0EE0FFF1FEE0FFF1F8E010F5F3C
:101C70001F4FD801AE0FBF1FEA5EFE4F15966D9144
:101C80007D918D919C911897278530894189528942
:101C90000E9413251B012C01E0913501F0E0EE0FAD
:101CA000FF1FEE0FFF1F0E0F1F1FEA5EFE4FD80132
:101CB00015966D917D918D919C911897278530890E
:101CC000418952890E9413253B014C018CE0FE01A1
:101CD0007296DF011D928A95E9F76F8D78A189A12F
:101CE0009AA120E030E040E850E40E94CD282F8DFA
:101CF00038A149A15AA10E94CD287B018C01C201C3
:101D0000B101A20191010E94CD289B01AC01C80143
:101D1000B7010E9413257B018C01C401B301A4010A
:101D200093010E94CD289B01AC01C801B7010E941C
:101D300013250E945A297B018C01C201B101A40123
:101D400093010E9408289B01AC0117FB109517F91D
:101D50001095C801B7010E94F4256B017C01A70111
:101D600096010E94AE29882321F084E08093160119
:101D7000D8C080911701833021F4F7FAF094F7F876
:101D8000F0946F8D78A189A19AA120E030E040E025
:101D900050E00E94ED2588236CF4F7FAF094F7F8F0
:101DA000F0944F8D58A169A17AA170584F8F58A314
:101DB00069A37AA300913401A02EBB24AA0CBB1CFA
:101DC000AA0CBB1C8E010F5F1F4FA00EB11EC401D9
:101DD000B301A70196010E94CD289B01AC01C2016D
:101DE000B1010E94132520E030E040E05FE30E9453
:101DF000CD28D50151966D937D938D939C935497E7
:101E00008091350190E0880F991F880F991F080F66
:101E1000191FC201B101A70196010E94CD289B01A3
:101E2000AC01C401B3010E94142520E030E040E081
:101E30005FE30E94CD28F801618B728B838B948BBA
:101E400015C0E0913501F0E0EE0FFF1FEE0FFF1F10
:101E5000EC0FFD1F2289338944895589C701B601DA
:101E60000E9408286F8F78A389A39AA390911701E5
:101E70002091340100913501E090360180901801E5
:101E8000882061F4F0911D01FDA340911E014EA335
:101E900050911F015FA36091200168A700D000D07E
:101EA0000F92EDB7FEB731964F8D58A169A17AA177
:101EB000ADB7BEB711964D935D936D937C93149718
:101EC00080E0923009F481E0848385E291E0BE01F4
:101ED0006A5F7F4FAE014E5E5F4FADA0BEA0CFA048
:101EE000D8A40E94C7040F900F900F900F900F90EE
:101EF000809116018823A9F4A5E2B1E0FE0136968F
:101F00008CE001900D928150E1F780911B018823B4
:101F100031F00E94B2221092E00510921B018091D4
:101F20001601A8960FB6F894DEBF0FBECDBFCF91B5
:101F3000DF911F910F91FF90EF90DF90CF90BF90B6
:101F4000AF909F908F907F906F905F904F903F9059
:101F50002F900895CA80DB80EC80FD80C701B60118
:101F60000E94A7290E945C269B01173409F4E9C846
:101F70001D3409F051CA01CA123509F4F9CA1335E2
:101F800084F41C343CF419340CF0C0CA163409F043
:101F900087CB81CA1C3409F4DCCA103509F080CB28
:101FA000E2CA183509F432CB19353CF4133509F47B
:101FB000FBCA143509F074CB10CB193509F43FCBAB
:101FC0001A3509F06DCB54CB10923701249A259A1B
:101FD0002C9808952C980895CF93DF93EC0180916D
:101FE000370190E0C817D90779F00E94B2222097F4
:101FF00041F01C161D0614F42D9801C02D9A2C9A40
:1020000001C02C98C0933701DF91CF910895EF92D2
:10201000FF920F931F937B018C0122E030E040E0A0
:1020200050E00E940B2A205C3D4B404F5F4FCA019D
:10203000B901A80197010E940B2A2150304030932A
:10204000C5002093C400E0ECF0E080818D7F8083A8
:10205000E1ECF0E080818061808380818860808312
:102060008081806880831F910F91FF90EF90089589
:10207000282FE0913A019E2F9F5F903431F490E039
:1020800004C08091070684FD0FC080913B01981722
:10209000C1F3F0E0E857F94F208390933A01809123
:1020A000C10080628093C10008951F920F920FB605
:1020B0000F9211248F939F93EF93FF9380913B0195
:1020C000E82FF0E0E857F94F90819093C600982FE1
:1020D0009F5F903409F490E090933B0180913A0126
:1020E000981729F48091C1008F7D8093C100FF91E2
:1020F000EF919F918F910F900FBE0F901F901895A9
:102100009091390180913801891711F4EFEF0DC0DA
:10211000E92FF0E0E85FF94FE081892F8F5F80932E
:102120003901803811F4109239018E2F0895809171
:1021300038018093390108951F920F920FB60F92C4
:1021400011242F933F934F935F936F937F938F93BC
:102150009F93AF93BF93EF93FF932091C6002132DB
:10216000A1F0223218F4283101F513C02F3319F0F1
:102170002E37D9F404C080910706816003C0809196
:10218000070682608093070621C080910706886059
:10219000F9CF8091070684FD04C00E94D9120E94E5
:1021A000EA0F809107068061EDCFE09138019E2F04
:1021B0009F5F903809F490E080913901981731F0D1
:1021C000F0E0E85FF94F208390933801FF91EF91A1
:1021D000BF91AF919F918F917F916F915F914F913F
:1021E0003F912F910F900FBE0F901F9018958BE687
:1021F00091E00E94F8248AE491E00E94F824109271
:102200006E0110926F010895CF93DF93EC01009758
:1022100019F485E491E036C08DE391E00E94F82442
:10222000C330D105D1F0C430D1053CF4C130D10563
:1022300071F0C230D105E9F40DC0C530D10599F077
:10224000C530D1056CF0C630D10599F40FC089E2D4
:1022500091E018C08FE091E015C087EF90E012C0C8
:1022600080EE90E00FC088EC90E00CC086EB90E030
:1022700009C0BE01882777FD8095982F0E94AB2466
:1022800083EB90E00E94F824DF91CF910895FC0148
:102290008081843221F4CF010E94B31A0895CF01C6
:1022A0000E9463080895DF93CF93CDB7DEB72C97D4
:1022B0000FB6F894DEBF0FBECDBFDE011196E1EE82
:1022C000F5E08CE001900D928150E1F780E091E023
:1022D0000E94062569817A818B819C810E948F26CC
:1022E0002091C8063091C9064091CA065091CB068C
:1022F0000E94F4250E943C2487E091E00E9406257C
:102300006D817E818F8198850E948F262091CC06D9
:102310003091CD064091CE065091CF060E94F42513
:102320000E943C2487E091E00E94062569857A8519
:102330008B859C850E948F262091D0063091D106F6
:102340004091D2065091D3060E94F4250E943C246D
:1023500089E091E00E94062569817A818B819C81C8
:102360000E948F262091C8063091C9064091CA0666
:102370005091CB060E94F4252091ED0530E0F90143
:10238000EE0FFF1FE20FF31FEE0FFF1FEE0FFF1FF9
:10239000E252FA4F20893189428953890E941325DC
:1023A0002091FA053091FB054091FC055091FD0507
:1023B0000E9413250E943C2487E091E00E9406259C
:1023C0006D817E818F8198850E948F262091CC0619
:1023D0003091CD064091CE065091CF060E94F42553
:1023E0002091ED0530E0F901EE0FFF1FE20FF31F22
:1023F000EE0FFF1FEE0FFF1FE252FA4F24893589BF
:10240000468957890E9413252091FE053091FF05CA
:1024100040910006509101060E9413250E943C2421
:1024200087E091E00E94062569857A858B859C85E9
:102430000E948F262091D0063091D1064091D2067D
:102440005091D3060E94F4252091ED0530E0F9016A
:10245000EE0FFF1FE20FF31FEE0FFF1FEE0FFF1F28
:10246000E252FA4F208D318D428D538D0E941325FB
:102470002091020630910306409104065091050612
:102480000E9413250E943C2482E191E00E940625CF
:102490002C960FB6F894DEBF0FBECDBFCF91DF9163
:1024A00008951F9380910706882381F18091070684
:1024B000182F84FF04C081E08093DE0527C080FFD1
:1024C00007C00E945311809107068E7F80930706F4
:1024D00013FF07C00E94D11380910706877F809366
:1024E000070612FF07C00E94DF13809107068B7F4B
:1024F0008093070611FF0AC00E94AC1381E080930D
:10250000E005809107068D7F809307061F9108954F
:102510001F9311E046C02A3011F02D30E1F40E94E3
:1025200051128091DE05882309F041C0E0916E01CF
:10253000EE2351F0F0E0E45CFE4F10828CE391E07A
:102540000E94471190E002C080E090E00E940411D8
:1025500010926E0106C080916F01882329F0293204
:1025600001F510926F011DC02132D8F02F32C9F051
:10257000283219F410936F0114C090916E019133B9
:1025800080F4822F8156E92FF0E09F5F8A3120F49A
:10259000E45CFE4F205202C0E45CFE4F2083909327
:1025A0006E010E948010282F8F3F09F0B4CF1F9139
:1025B000089580916F008D7F80936F008AEF90E087
:1025C00020E931E0F9013197F1F70197D9F7289A1D
:1025D00008951F920F920FB60F9211248F939F931D
:1025E0009BB18091DE068C71937E892B8BB9109202
:1025F000B1009F918F910F900FBE0F901F90189573
:102600008AB18C6F8AB98BB183709091DE06892B69
:102610008BB9209A809181008F7E80938100809178
:102620008100886080938100809180008D7F8093FD
:102630008000809180008E7F809380008091800058
:102640008F7380938000809180008F7C80938000C6
:102650001092B0001092B100809170008160809360
:10266000700080916F008D7F80936F008AEF90E003
:1026700020E931E0F9013197F1F70197D9F7289A6C
:1026800008959B01AC01203283E0380780E04807C1
:1026900080E0580720F420E233E040E050E060E0C2
:1026A00070E788E399E30E94E929C901DA018030E3
:1026B00020E0920721E0A20720E0B20738F4FC01F5
:1026C0009C0140E050E060E070E031C0803020E0EC
:1026D000920728E0A20720E0B207A8F473E0B695BD
:1026E000A795979587957A95D1F7FC019C0140E0D5
:1026F00050E063E0220F331F441F551F6A95D1F746
:1027000061E070E014C026E0B695A795979587958F
:102710002A95D1F7FC019C0140E050E086E0220FB1
:10272000331F441F551F8A95D1F762E070E08091F6
:102730008100962F9F5F887F982B90938100F09364
:102740008900E093880020938401309385014093B1
:10275000860150938701089580910606882301F52C
:102760008091DF058823E1F481E080930606809163
:10277000DE06809397018091D50690E0A0E0B0E05E
:102780000297A109B109880F991FAA1FBB1F819544
:1027900080939601289880916F00826080936F00EB
:1027A00008958091DF05882349F4809106068823E7
:1027B00029F01092E00581E08093DF050895E09113
:1027C0009401F09195013097A1F165857685878513
:1027D0009089209180013091810140918201509136
:1027E0008301621B730B840B950B0E94771E109262
:1027F0008C0110928D0110928E0110928F0160E079
:1028000070E080E090E00E94411380E091E7A2E058
:10281000B0E08093880190938901A0938A01B093DE
:102820008B0110928001109281011092820110920E
:1028300083011092DF05089584E2E0E7F1E0DF0113
:102840001D928A95E9F760E273E080E090E00E94D3
:1028500041131092950110929401109298010895DD
:102860001F920F920FB60F921124EF92FF920F93C7
:102870001F932F933F934F935F936F937F938F9308
:102880009F93AF93BF93CF93DF93EF93FF93809189
:102890009801882309F06AC39BB120919701822F88
:1028A000807E9F71892B8BB98BB1837E822B8BB9F4
:1028B000809196018093B20082E08093B10081E024
:1028C0008093980178948091940190919501892B3F
:1028D00009F08EC00E94231BEC0190939501809318
:1028E0009401009709F46EC08091DF058823D1F42C
:1028F0006BA17CA18DA19EA160938C0170938D0131
:1029000080938E0190938F010E94411380E091E7A4
:10291000A2E0B0E08093880190938901A0938A019E
:10292000B0938B012BA53CA54DA55EA5DA01C9018D
:10293000B595A79597958795820F931FA41FB51FEF
:102940008093900190939101A0939201B093930191
:102950002D853E854F855889DA01C901B595A79522
:1029600097958795B095A095909581959F4FAF4F7E
:10297000BF4F8093700190937101A0937201B09347
:1029800073018093740190937501A0937601B093C5
:1029900077018093780190937901A0937A01B093A5
:1029A0007B0120937C0130937D0140937E01509305
:1029B0007F01109280011092810110928201109289
:1029C000830116C080916F008D7F80936F008AEF26
:1029D00090E020E931E0F9013197F1F70197D9F75B
:1029E000289A109206068091070684608093070655
:1029F000E0919401F0919501309709F4AEC22081E5
:102A00002093970140917001509171016091720182
:102A10007091730181819281A381B481480F591F04
:102A20006A1F7B1F40937001509371016093720184
:102A3000709373011416150616061706C4F5246064
:102A40002093970180917C0190917D01A0917E015E
:102A5000B0917F01481B590B6A0B7B0B40937001AF
:102A600050937101609372017093730125FF0CC044
:102A70008091E1059091E205A091E305B091E40514
:102A80000197A109B1090BC08091E1059091E20580
:102A9000A091E305B091E4050196A11DB11D8093BD
:102AA000E1059093E205A093E305B093E40540911E
:102AB0007401509175016091760170917701858163
:102AC0009681A781B085480F591F6A1F7B1F4093CD
:102AD0007401509375016093760170937701141619
:102AE000150616061706D4F5209197012860209345
:102AF000970180917C0190917D01A0917E01B09120
:102B00007F01481B590B6A0B7B0B40937401509358
:102B10007501609376017093770126FF0CC0809158
:102B2000E5059091E605A091E705B091E8050197CC
:102B3000A109B1090BC08091E5059091E605A0912E
:102B4000E705B091E8050196A11DB11D8093E5054B
:102B50009093E605A093E705B093E80540917801CE
:102B60005091790160917A0170917B018185928504
:102B7000A385B485480F591F6A1F7B1F40937801B6
:102B80005093790160937A0170937B0114161506B6
:102B900016061706D4F5209197012061209397011E
:102BA00080917C0190917D01A0917E01B0917F0187
:102BB000481B590B6A0B7B0B4093780150937901AA
:102BC00060937A0170937B0127FF0CC08091E90527
:102BD0009091EA05A091EB05B091EC050197A10950
:102BE000B1090BC08091E9059091EA05A091EB0530
:102BF000B091EC050196A11DB11D8093E90590935C
:102C0000EA05A093EB05B093EC052091800130918B
:102C1000810140918201509183012F5F3F4F4F4FBF
:102C20005F4F209380013093810140938201509344
:102C3000830185859685A785B089281739074A07B6
:102C40005B0708F084C18091DF05882309F46AC01E
:102C50002091840130918501409186015091870136
:102C60008091880190918901A0918A01B0918B0196
:102C7000280F391F4A1F5B1F209388013093890159
:102C800040938A0150938B01213002EE300704E01B
:102C9000400700E0500708F460C12050324E444025
:102CA0005040209388013093890140938A015093CA
:102CB0008B0120918C0130918D0140918E015091BA
:102CC0008F0163A574A585A596A562177307840770
:102CD0009507B8F080916F008D7F80936F008AEF29
:102CE00090E020E931E0F9013197F1F70197D9F748
:102CF000289A109206068091070684608093070642
:102D00002CC179018A01E61AF70A080B190BC801D0
:102D1000B701E0928C01F0928D0100938E01109327
:102D20008F016CC087A590A9A1A9B2A9281739075E
:102D30004A075B0708F065C0209184013091850146
:102D4000409186015091870180918801909189017D
:102D5000A0918A01B0918B01280F391F4A1F5B1F78
:102D6000209388013093890140938A0150938B010D
:102D7000213002EE300704E0400700E0500708F47D
:102D8000ECC02050324E4440504020938801309394
:102D9000890140938A0150938B0183A594A5A5A531
:102DA000B6A520918C0130918D0140918E015091FA
:102DB0008F01820F931FA41FB51F80938C019093E6
:102DC0008D01A0938E01B0938F0127A930AD41AD45
:102DD00052AD82179307A407B50740F020938C01EA
:102DE00030938D0140938E0150938F0160918C013F
:102DF00070918D0180918E0190918F010E944113FD
:102E0000ACC083A994A9A5A9B6A9281739074A0770
:102E10005B0708F480C0281739074A075B0769F485
:102E200080E091E7A2E0B0E080938801909389016F
:102E3000A0938A01B0938B0190C0209184013091BE
:102E40008501409186015091870180918801909180
:102E50008901A0918A01B0918B01280F391F4A1F67
:102E60005B1F209388013093890140938A0150931E
:102E70008B01213012EE310714E0410710E05107B9
:102E800008F46BC02050324E4440504020938801DB
:102E90003093890140938A0150938B0120918C01DA
:102EA00030918D0140918E0150918F018091900160
:102EB00090919101A0919201B09193018217930793
:102EC000A407B50748F483A594A5A5A5B6A5281B16
:102ED000390B4A0B5B0B04C05695479537952795E0
:102EE00020938C0130938D0140938E0150938F017C
:102EF00027A130A541A552A580918C0190918D010B
:102F0000A0918E01B0918F0182179307A407B50796
:102F100008F06CCF63CF27A930AD41AD52AD8091A1
:102F20008C0190918D01A0918E01B0918F0182173B
:102F30009307A407B50789F020938C0130938D0186
:102F400040938E0150938F01CA01B90157CF10925F
:102F50009501109294010E94141B80919701909109
:102F6000DE0689278093970110929801FF91EF91D7
:102F7000DF91CF91BF91AF919F918F917F916F9191
:102F80005F914F913F912F911F910F91FF90EF9083
:102F90000F900FBE0F901F901895F999FECF92BD1C
:102FA00081BD81E08FBB80B50895F894F999FECF7B
:102FB00092BD81BD81E08FBB40B54627842F992704
:102FC00087FD9095262F30E082239323892B39F0BB
:102FD0006F3F19F060BD84E006C084E104C0442363
:102FE00021F060BD84E28FBBF99A789408958F92A6
:102FF0009F92AF92BF92CF92DF92EF92FF920F9388
:10300000DF93CF9300D0CDB7DEB75C016B017A01BF
:103010004A0100E01EC0002319F021E030E008C0A2
:10302000202F332727FD30952227330F221F3327E8
:10303000F60161916F01062F020F9C012F5F3F4F38
:103040003A8329830E94D5170894810891088981C1
:103050009A8181149104F9F6C7018A0D9B1D602F96
:103060000E94D5170F900F90CF91DF910F91FF9095
:10307000EF90DF90CF90BF90AF909F908F9008958A
:10308000CF93DF93EC01FB019A0190E0B1E019C00E
:10309000F999FECFF2BDE1BDBFBBA0B5992319F0F0
:1030A00081E090E008C0892F992787FD90958827B7
:1030B000990F881F992731969A2F980FA99321501D
:1030C00030402115310521F7460F571FF999FECFE2
:1030D00052BD41BD81E08FBB80B520E030E0981744
:1030E00011F421E030E0C901DF91CF91089580E033
:1030F00090E064E00E94D51781E090E068EC76E013
:1031000043E250E00E94F7170895EF92FF920F9369
:103110001F93CF93DF93EC017A018B0185309105EA
:1031200009F455C08630910554F48330910581F13E
:10313000843091050CF042C097FF12C086C08730E2
:10314000910509F456C0873091050CF449C08830C8
:10315000910509F457C08930910509F076C069C01E
:10316000CB01BA0120E030E040E050E00E94ED25C4
:1031700018161CF082E092E06FC0CC0FDD1FCC0F60
:10318000DD1FC853D94FE882F9820A831B8360C0D0
:10319000CB01BA0120E030E040E450E40E94ED258C
:1031A00088231CF48BED91E057C0C801B7010E9441
:1031B00030290E9461266093D5064AC04093D60606
:1031C0005093D7066093D8067093D90641C04093B8
:1031D000DA065093DB066093DC067093DD0638C098
:1031E0004093DF065093E0066093E1067093E20699
:1031F0002FC0CB01BA010E94A7290E9461266093CB
:10320000DE0626C0CB01BA0120E030E040E752E400
:103210000E94CD2820E030E040E752E40E94CD2813
:103220006093E3067093E4068093E5069093E606C8
:103230000FC0DB01CA01BF778093E7069093E806D1
:10324000A093E906B093EA0603C087EC91E004C0BE
:103250000E94771882EB91E00E94F824DF91CF91D1
:103260001F910F91FF90EF9008951F9380E090E0E1
:103270000E94CD17182F843081F488EC96E061E02D
:1032800070E043E250E00E94401820E0892B09F4EE
:1032900021E081E0282730E05EC0813021F588EC14
:1032A00096E061E070E04BE150E00E944018892B0D
:1032B00009F44FC080E098ECAFE2B8E48093E306F5
:1032C0009093E406A093E506B093E6068DEC9CECA3
:1032D000ACE4BDE38093E7069093E806A093E9068B
:1032E000B093EA0631C08250823098F588EC96E0BF
:1032F00061E070E043E250E00E944018892B49F100
:10330000123061F48DEC9CECACE4BDE38093E706F5
:103310009093E806A093E906B093EA066091E3066D
:103320007091E4068091E5069091E60620E030E099
:1033300041E655E40E94CD286093E3067093E406CD
:103340008093E5069093E6060E94771821E030E02E
:1033500002C020E030E0C9011F91089585E993E0A3
:103360000E94F8246091C8067091C9068091CA062F
:103370009091CB060E943C2480E893E00E94F824C0
:103380006091CC067091CD068091CE069091CF06CB
:103390000E943C248BE693E00E94F8246091D006C2
:1033A0007091D1068091D2069091D3060E943C2460
:1033B00086E593E00E94F8246091D50670E080E0F5
:1033C00090E00E94AB2484E393E00E94F824609193
:1033D000D6067091D7068091D8069091D9060E94A2
:1033E0003C2481E193E00E94F8246091DA06709118
:1033F000DB068091DC069091DD060E943C248EEE77
:1034000092E00E94F8246091DF067091E0068091BE
:10341000E1069091E2060E943C2485ED92E00E9434
:10342000F8246091DE0670E080E090E00E94AB241A
:1034300082EB92E00E94F8248091DE060E94C7246D
:1034400089EA92E00E94F8246091E3067091E40614
:103450008091E5069091E60620E030E041E655E4F3
:103460000E94F4250E943C2486E892E00E94F82401
:103470006091E7067091E8068091E9069091EA066E
:103480000E943C2480E692E00E94F8248BE192E0C6
:103490000E94F82408950E943519892B09F062C012
:1034A00087E791E00E94F82484EF99EFACE3B4E45D
:1034B0008093C8069093C906A093CA06B093CB0622
:1034C0008093CC069093CD06A093CE06B093CF0602
:1034D0008093D0069093D106A093D206B093D306E2
:1034E0008EE18093D50680E090E0AAEFB3E480936C
:1034F000D6069093D706A093D806B093D9068093AA
:10350000DA069093DB06A093DC06B093DD0680E03C
:1035100098ECAFE2B8E48093E3069093E406A093BE
:10352000E506B093E6068DEC9CECACECBDE3809335
:10353000DF069093E006A093E106B093E2068CE1EB
:103540008093DE068DEC9CECACE4BDE38093E70653
:103550009093E806A093E906B093EA060E947718D4
:103560000E94AE190895EF92FF920F931F93DF937D
:10357000CF93CDB7DEB729970FB6F894DEBF0FBE55
:10358000CDBF8C0181E08983F80180818432E1F52F
:103590008181882319F40E94AE1934C0C8017E01CC
:1035A0000894E11CF11CB701AE014E5F5F4F0E9411
:1035B000F622892B59F19981F801E90FF11D8081DB
:1035C0008D3311F59F5F9983C801B701AE014A5F42
:1035D0005F4F0E94F622892BC9F08981080F111DC7
:1035E000F8018081882381F46A817B818C819D81AF
:1035F0000E945C26DC01CB014E815F816885798564
:103600000E94851880E003C083E001C081E0299614
:103610000FB6F894DEBF0FBECDBFCF91DF911F91E3
:103620000F91FF90EF9008959091BF058091C00594
:10363000981741F08091C0058F5F823109F480E0D6
:103640008093C00508959091BF058091C00598179B
:1036500019F420E030E008C09091C0058BE3989FFA
:103660009001112427563E4FC90108959091C0053D
:1036700020E08091C105981709F421E0822F089578
:10368000EF92FF920F931F936093C2057093C3054F
:103690008093C4059093C5052093C6053093C70554
:1036A0004093C8055093C905E092CA05F092CB0536
:1036B0000093CC051093CD051F910F91FF90EF90D3
:1036C00008958F929F92AF92BF92CF92DF92EF9226
:1036D000FF920F931F93CF93DF93EC016B01009741
:1036E00009F460C08AA1882309F05CC0ED88FE88D7
:1036F0000F89188DFB01B588A6889788808CC80132
:10370000B7012B2D3A2D492D582D0E94ED258823E8
:103710000CF048C0C801B701A80197010E94CD284C
:103720007B018C016091E3067091E4068091E506CF
:103730009091E606905820E030E040E050EC0E9486
:10374000CD282D8D3E8D4F8D58A10E94CD289B01F7
:10375000AC01C801B7010E9414250E945A297B01BF
:103760008C016B2D7A2D892D982D9701A8010E942F
:10377000ED25882324F4EB2CFA2C092D182D6B2D24
:103780007A2D892D982D9701A8010E94ED25882377
:1037900049F0C701D801F601858B968BA78BB08FB6
:1037A00081E081A3DF91CF911F910F91FF90EF9066
:1037B000DF90CF90BF90AF909F908F9008952F9201
:1037C0003F924F925F926F927F928F929F92AF92B1
:1037D000BF92CF92DF92EF92FF920F931F93DF93EE
:1037E000CF93CDB7DEB768970FB6F894DEBF0FBEA4
:1037F000CDBF1C016A017B0128013901DC01D7968C
:103800006D917D918D919C91DA970E948D264B014F
:103810005C01A70196010E94CD280E94DA250E9432
:1038200061267B018C01F10163A374A385A396A398
:10383000C501B401A30192010E94CD280E94DA259E
:103840000E94612669877A878B879C87D10197962A
:103850006D937D938D939C939A979B966D917D919B
:103860008D919C919E9722E330E040E050E00E94D1
:10387000CA290E948F2620E030E040E752E40E94EF
:10388000CD280E945C262B013C01C801B7010E9493
:103890008D267B018C01C301B2010E948F266D83AE
:1038A0007E838F839887C501B401A50194010E948E
:1038B000CD285B016C01C801B701A80197010E94E6
:1038C000CD286D877E878F87988B6D817E818F81D4
:1038D00098859B01AC010E941425698B7A8B8B8B98
:1038E0009C8BC601B5012D853E854F8558890E9468
:1038F000132529893A894B895C890E94F4250E9405
:10390000DA250E945C2669837A838B839C83698590
:103910007A858B859C850E948D269B01AC010E9437
:10392000CD286D8B7E8B8F8B988FA60195010E9481
:1039300013257B018C017094609450944094411C39
:10394000511C611C711CC301B2010E948F269B0196
:10395000AC010E9414259B01AC01C801B7010E9473
:10396000F4250E94CA26F101A584B684C784D088B4
:103970008601750129813A814B815C81E21AF30A43
:10398000040B150B0E945C26A8019701261B370B20
:10399000480B590BDA01C90157FF4AC0C601B501EE
:1039A0000E948F269B01AC0169897A898B899C8949
:1039B0000E94CD282D853E854F8558890E9413256C
:1039C0002D893E894F89588D0E9414257B018C01D9
:1039D0006D817E818F81988520E030E040E850E461
:1039E0000E94CD289B01AC01C801B7010E94F425BB
:1039F0000E94DA250E945C26AC01CB01DA01BC01F1
:103A0000CD0197FF04C060E070E080E090E0698342
:103A10007A838B839C83A616B706C806D90624F43E
:103A2000A982BA82CB82DC8280E090E0A0E0B0E0A4
:103A300029813A814B815C81F10127A730AB41ABF1
:103A400052AB820F931FA41FB51F83AB94ABA5ABE2
:103A5000B6AB68960FB6F894DEBF0FBECDBFCF9160
:103A6000DF911F910F91FF90EF90DF90CF90BF906B
:103A7000AF909F908F907F906F905F904F903F900E
:103A80002F9008952F923F924F925F927F928F9244
:103A90009F92AF92BF92CF92DF92EF92FF920F93DD
:103AA0001F93CF93DF93D090BF058091E306909151
:103AB000E406A091E506B091E6061C012D0157FA37
:103AC000509457F8509400E010E0C0E0D0E0BB24E0
:103AD000B3943BE3C32E72C0DD2011F422E1D22E59
:103AE000DA94209709F463C00115110509F45FC049
:103AF000A98C9A8C8B8C7C8C6D897E898F89988D12
:103B00002A2D392D482D572D0E94ED25882309F4A3
:103B10004EC08AA1882309F041C0F801E588F688E3
:103B20000789108D6A2D792D882D972DA801970171
:103B30000E94FB27181694F5C801B701A801970148
:103B40000E94CD287B018C01C201B10120E030E050
:103B500040E050EC0E94CD282D8D3E8D4F8D58A118
:103B60000E94CD289B01AC01C801B7010E94142519
:103B70000E945A29162F072FF82EE92E6A2D792D2B
:103B8000882D972D212F302F4F2D5E2D0E94ED2552
:103B900087FD04C0A12E902E8F2C7E2C8A2D992D6E
:103BA000A82DB72D8D8B9E8BAF8BB88FB9A2DC9CC7
:103BB000C00111248E01EC01C756DE4F8091C00573
:103BC000D81609F089CFF090C00520E030E000E081
:103BD00010E09BE3E92E11C0FE9CE0011124C756C2
:103BE000DE4FC901B801AE010E94611BF394F2E1FE
:103BF000FF1609F4FF2498018E018091BF05F81685
:103C000059F7C901B80140E050E00E94611B709073
:103C1000C005C0E0D0E08BE3582E35C0759C400154
:103C2000112489E991E0880E991E209731F189A12C
:103C3000882321F4F40181A18823F9F0E988FA8826
:103C40000B891C896D897E898F89988DA8019701C0
:103C50000E94F4255B016C01F401658976898789EE
:103C6000908DA80197010E94F4258B019C01CE0143
:103C7000B601A5010E94DF1B19A27394F2E17F1621
:103C800009F47724E4018091BF05781639F6E988B4
:103C9000FA880B891C896D897E898F89988DA80186
:103CA00097010E94F4255B016C0160E070E080E008
:103CB00090E0A80197010E94F4258B019C01CE01A0
:103CC000B601A5010E94DF1B19A2DF91CF911F91C0
:103CD0000F91FF90EF90DF90CF90BF90AF909F90AB
:103CE0008F907F905F904F903F902F900895AF926C
:103CF000BF92CF92DF92EF92FF920F931F93CF93D9
:103D0000DF935B016C019091C0058BE3989FE0010C
:103D10001124C756DE4FC601B5010E948F262D8D96
:103D20003E8D4F8D58A10E94CD287B018C016D8561
:103D30007E858F8598890E948F269B01AC01C801E2
:103D4000B7010E94F4256D8F7E8F8F8F98A3AD866B
:103D5000BE86CF86D88A80E090E0A0E0B0E08D8B70
:103D60009E8BAF8BB88F898F9A8FAB8FBC8F1AA227
:103D700081E089A30E94421DDF91CF911F910F9195
:103D8000FF90EF90DF90CF90BF90AF9008952F926B
:103D90003F924F925F926F927F928F929F92AF92DB
:103DA000BF92CF92DF92EF92FF920F931F93DF9318
:103DB000CF93CDB7DEB7C355D0400FB6F894DEBF72
:103DC0000FBECDBF29013A012396ACAEBDAECEAE3B
:103DD000DFAE239724968FAE24973091BF052BE357
:103DE000329FA001112447565E4F5A8F498F209170
:103DF000C8063091C9064091CA065091CB062BAF38
:103E00003CAF4DAF5EAF0E94CD280E949D28299601
:103E10006FAF29972A967FAF2A972B968FAF2B9754
:103E20002C969FAF2C978091CC069091CD06A091B7
:103E3000CE06B091CF068FAB98AFA9AFBAAFC30192
:103E4000B2012FA938AD49AD5AAD0E94CD280E94CC
:103E50009D282D966FAF2D972E967FAF2E972F967C
:103E60008FAF2F9760969FAF60972091D0063091CB
:103E7000D1064091D2065091D3062BAB3CAB4DAB53
:103E80005EABC801B7010E94CD280E949D286196B3
:103E90006FAF619762967FAF629763968FAF6397BC
:103EA00064969FAF6497A98DBA8D1C922091C2052C
:103EB0003091C3054091C4055091C5052C968CAD39
:103EC0009DADAEADBFAD2C9782179307A407B50784
:103ED00024F480E2A98DBA8D8C934090C605509051
:103EE000C7056090C8057090C90560968CAD9DAD02
:103EF000AEADBFAD609784159505A605B7052CF44A
:103F0000A98DBA8D8C9180648C93E090CA05F09055
:103F1000CB050091CC051091CD0564968CAD9DAD7F
:103F2000AEADBFAD64978E159F05A007B1072CF409
:103F3000A98DBA8D8C9180688C932C96ACACBDAC5D
:103F4000CEACDFAC2C97A21AB30AC40AD50AE98D0D
:103F5000FA8DA182B282C382D482D7FE0BC0882799
:103F60009927DC018A199B09AC09BD0981839283D9
:103F7000A383B48360962CAD3DAD4EAD5FAD60972D
:103F8000241935094609570939014A01A98DBA8D05
:103F900015962D933D934D935C93189757FF0DC045
:103FA00088279927DC01821B930BA40BB50BE98DA5
:103FB000FA8D85839683A783B08764962CAC3DAC3D
:103FC0004EAC5FAC64972E183F08400A510AA2011C
:103FD000910157FE07C022273327A901221933096F
:103FE00044095509A98DBA8D19962D933D934D938A
:103FF0005C931C971596ED90FD900D911C91189770
:10400000FD0181819281A381B4818E159F05A00756
:10401000B10710F4D801C70182179307A407B507A9
:1040200010F4DA01C901E98DFA8D85879687A78793
:10403000B08B0097A105B10509F47AC2C601B5019C
:104040000E948F262BAD3CAD4DAD5EAD0E94F42598
:104050006FA778AB89AB9AABC401B3010E948F26DE
:104060002FA938AD49AD5AAD0E94F4256BA77CA7A6
:104070008DA79EA7C201B1010E948F262BA93CA942
:104080004DA95EA90E94F4256FA378A789A79AA7D6
:104090006FA578A989A99AA99B01AC010E94CD2896
:1040A0007B018C016BA57CA58DA59EA59B01AC0118
:1040B0000E94CD289B01AC01C801B7010E941425C4
:1040C0007B018C016FA178A589A59AA59B01AC0104
:1040D0000E94CD289B01AC01C801B7010E941425A4
:1040E0000E945A297B018C01A98DBA8D5D966D9332
:1040F0007D938D939C93909760E070E080E89FE3C0
:10410000A80197010E94F4252B013C012496BFAD24
:104110002497BB2359F423966CAD7DAD8EAD9FAD36
:104120002397A30192010E94CD280CC060E070E0AB
:1041300080E89FE323962CAD3DAD4EAD5FAD239758
:104140000E94F4255B016C01C801B701A60195012D
:104150000E94CD2828966CAF7DAF8EAF9FAF289779
:10416000E98DFA8D618B728B838B948B6585768557
:10417000878590890E948F267B018C01A60195017D
:104180000E94CD280E94DA250E946126A98DBA8D51
:10419000D7966D937D938D939C93DA972091E30648
:1041A0003091E4064091E5065091E6062BA33CA32E
:1041B0004DA35EA3C801B701A30192010E94CD28BF
:1041C0002BA13CA14DA15EA10E94CD2820E030E8AA
:1041D0004BE355E40E94F4250E94DA250E945C26F8
:1041E000A98DBA8D9B966D937D938D939C939E978D
:1041F0006FA578A989A99AA9A30192010E94CD2847
:104200006F8F78A389A39AA36BA57CA58DA59EA586
:10421000A30192010E94CD286B8F7C8F8D8F9E8F82
:104220006FA178A589A59AA5A30192010E94CD2826
:104230001B012C019091BF058091C005981709F4CE
:10424000B7C06090DA057090DB058090DC05909037
:10425000DD05B301C40120E030E040E050E00E9401
:10426000FB2718160CF0A4C06091CE057091CF0505
:104270008091D0059091D10590582F8D38A149A1FA
:104280005AA10E94CD287B018C016B8D7C8D8D8D78
:104290009E8D2091D2053091D3054091D405509147
:1042A000D5050E94CD289B01AC01C801B7010E9431
:1042B00013257B018C01C201B1012091D6053091FB
:1042C000D7054091D8055091D9050E94CD289B0172
:1042D000AC01C801B7010E9413257B018C0123E3C7
:1042E00033E343E75FE30E94ED2588230CF060C0D1
:1042F000B301C40128962CAD3DAD4EAD5FAD2897FE
:104300000E94ED2587FD08C028968CAD9DADAEAD11
:10431000BFAD28973C014D01C801B70123E333E34A
:1043200043E75FEB0E94FB2718160CF046C060E0E5
:1043300070E080E89FE3A80197010E94132520E028
:1043400030E040E05FE30E94CD280E945A295B01E3
:104350006C016BA17CA18DA19EA12091E7063091FB
:10436000E8064091E9065091EA060E94CD28A60190
:1043700095010E94CD287B018C0160E070E080E80F
:104380009FE3A60195010E9413259B01AC01C80182
:10439000B7010E94F4250E945A297B018C01B301C8
:1043A000C4019701A8010E94ED2587FD06C007C042
:1043B000EE24FF2400E010E002C073018401C70175
:1043C000D801E98DFA8D818F928FA38FB48F6BA165
:1043D0007CA18DA19EA1905820E030E040E050ECFF
:1043E0000E94CD28A98DBA8D5D962D913D914D915C
:1043F0005C9190970E94CD2820E030E040E050E0B2
:104400000E9414250E945A29D62EC72EB82EA92EF6
:10441000B701C8012D2D3C2D4B2D5A2D0E94ED25A5
:1044200087FD04C0ED2CFC2C0B2D1A2DC701D801E3
:10443000E98DFA8D858B968BA78BB08F61897289F8
:10444000838994892D2D3C2D4B2D5A2D0E94ED25CD
:10445000181634F081E0A98DBA8D92968C9303C022
:10446000E98DFA8D12A281E0A98DBA8D91968C9377
:104470002D8A3E8A4F8A588E2B8D3C8D4D8D5E8DB8
:10448000298B3A8B4B8B5C8B8F8D98A1A9A1BAA1FC
:104490008D879E87AF87B88B64962CAD3DAD4EADB2
:1044A0005FAD649729873A874B875C8760968CADB0
:1044B0009DADAEADBFAD60978D839E83AF83B88752
:1044C0002C962CAD3DAD4EAD5FAD2C9729833A8334
:1044D0004B835C83AEECB5E0FE013D968CE0019031
:1044E0000D928150E1F7E98DFA8D81899289A38936
:1044F000B4898093DA059093DB05A093DC05B09333
:10450000DD058091C1058093BF058091BF058F5F58
:10451000823109F480E08093C105A2ECB5E0FE0190
:1045200031968CE001900D928150E1F70E94421D7E
:10453000CD5ADF4F0FB6F894DEBF0FBECDBFCF917F
:10454000DF911F910F91FF90EF90DF90CF90BF9080
:10455000AF909F908F907F906F905F904F903F9023
:104560002F9008951F931BE306C00E945112809163
:10457000DE05882391F49091BF058091C0059817BE
:1045800041F08091C005819FC001112487569E4F44
:1045900061F780910606882341F71F910895809165
:1045A000BF058093C0058091BF058F5F823109F4FC
:1045B00080E08093C1058CE1E2ECF5E0DF011D9223
:1045C0008A95E9F7089520EA3FE004C0F9013197A0
:1045D000F1F701970097D1F7089535E004C0232F34
:1045E0002A95F1F701970097D1F70895AF92BF92FE
:1045F000CF92DF92EF92FF920F931F93DF93CF93AF
:1046000000D0CDB7DEB76C015B017A01FB01808180
:104610008601080F111DC801BE016F5F7F4F0E9408
:104620000A02F701608371838283938389819A816F
:104630008017910719F420E030E005C08C19F501CE
:10464000808321E030E0C9010F900F90CF91DF917E
:104650001F910F91FF90EF90DF90CF90BF90AF90A0
:10466000089584B1817F84B908956F927F928F926B
:104670009F92AF92BF92CF92DF92EF92FF920F93F1
:104680001F93982EA62EB42E670178018091D5062F
:10469000C81AD108E108F108992011F094EE01C080
:1046A00090EEA1109860B1109061222311F080EE7D
:1046B00098270091DE0609278BB1902F907E8F718D
:1046C000982B9BB924E0622E98E0792E80E1882E09
:1046D00083B1992021F0199902C006259924AA20B6
:1046E00021F01A9902C00725AA24BB2021F01B99AA
:1046F00002C00825BB24992021F4AA2011F4BB2074
:1047000089F08BB1102F1C71812B8BB98091D5064C
:1047100090E00E94ED228BB118271BB9C6010E94C0
:10472000ED22D6CF1F910F91FF90EF90DF90CF90A9
:10473000BF90AF909F908F907F906F900895DF9281
:10474000EF92FF920F931F930E94B222D3B080E0AA
:1047500060E041E020E0F0EAEF2EF6E8FF2EF1E025
:104760000F2F112D0E94352381E061E040E020E011
:104770000E94352383B18D258E7090E0BC01769523
:104780006795769567956170AC0173E0569547958E
:104790007A95E1F7417096958795817021E030E236
:1047A000E32E31EAF32E37E0032F112D0E9435233B
:1047B0001F910F91FF90EF90DF900895AF92BF92FD
:1047C000CF92DF92EF92FF920F93DF93CF93CDB70B
:1047D000DEB7A2970FB6F894DEBF0FBECDBF6B0158
:1047E0007C01611571058105910521F480E30E942A
:1047F000381032C000E05E010894A11CB11CC50154
:10480000800F911D9AA389A3C701B6012AE030E069
:1048100040E050E00E94E929E9A1FAA160830F5F1E
:10482000C701B6012AE030E040E050E00E94E929EB
:10483000C901DA016C017D01C114D104E104F10464
:10484000F1F608C0FE01E00FF11D8081805D0E943D
:10485000381001500023B1F7A2960FB6F894DEBFCE
:104860000FBECDBFCF91DF910F91FF90EF90DF9002
:10487000CF90BF90AF900895AF92BF92CF92DF924A
:10488000EF92FF920F931F93CF93DF937B018C01E5
:1048900020E030E040E050E00E94ED2588233CF429
:1048A0008DE20E94381017FB109517F91095C8017A
:1048B000B7012AE037ED43EA5BE30E9414257B0150
:1048C0008C010E945C265B016C01CC24B7FCC09477
:1048D000DC2CC601B5010E94DE238EE20E94381056
:1048E000C601B5010E948F269B01AC01C801B7012A
:1048F0000E941325C2E0D0E01EC020E030E040E27C
:1049000051E40E94CD285B016C010E945C267B0172
:104910008C01862F805D0E9438106E2D70E08827F4
:1049200077FD8095982F0E948F269B01AC01C601D0
:10493000B5010E94132521972FEFCF3FD207E9F64B
:10494000DF91CF911F910F91FF90EF90DF90CF906B
:10495000BF90AF900895EF92FF920F931F937B014A
:104960008C0197FF0BC08DE20E94381010950095C6
:10497000F094E094E11CF11C011D111DC801B70168
:104980000E94DE231F910F91FF90EF9008950F93E7
:104990001F93DF93CF93CDB7DEB728970FB6F89468
:1049A000DEBF0FBECDBF982FFE0131969E01275F5F
:1049B0003F4F892F817081939695E217F307C9F7CE
:1049C0008E01085F1F4FF8018081805D0E943810C2
:1049D000015010400C171D07B1F728960FB6F89438
:1049E000DEBF0FBECDBFCF91DF911F910F91089514
:1049F000CF93DF93EC0102C00E943810FE01219694
:104A000084918823C9F7DF91CF910895CF93DF93E5
:104A1000EC0103C021960E94381088818823D1F7C9
:104A2000DF91CF9108955058BB27AA270ED081C29D
:104A300041D230F046D220F031F49F3F11F41EF401
:104A400011C20EF4E095E7FBDCC1E92F94D280F3AC
:104A5000BA17620773078407950718F071F49EF57B
:104A6000C3C20EF4E0950B2EBA2FA02D0B01B90195
:104A700090010C01CA01A0011124FF27591B99F0D4
:104A8000593F50F4503E68F11A16F040A22F232FE0
:104A9000342F4427585FF3CF469537952795A79530
:104AA000F0405395C9F77EF41F16BA0B620B730BD7
:104AB000840BBAF09150A1F0FF0FBB1F661F771F48
:104AC000881FC2F70EC0BA0F621F731F841F48F4FD
:104AD000879577956795B795F7959E3F08F0B3CF83
:104AE0009395880F08F09927EE0F9795879508956D
:104AF000E1D158F080E891E009F49EEFE2D128F08E
:104B000040E851E059F45EEF09C0ACC16DC2E92F35
:104B1000E07831D268F3092E052AC1F3261737074A
:104B20004807590738F00E2E07F8E02569F0E02510
:104B3000E0640AC0EF6307F8009407FADB01B901EB
:104B40009D01DC01CA01AD01EF935DD0F2D10AD025
:104B50005F91552331F02BED3FE049E450FD49ECE6
:104B600063CF0895DF93DD27B92FBF7740E85FE378
:104B70001616170648075B0710F4D92FA1D29F938A
:104B80008F937F936F93E0D3E8E6F0E06ED1D1D1BD
:104B90002F913F914F915F910CD3DD2349F09058B5
:104BA000A2EA2AED3FE049EC5FE3D0785D274DDFD4
:104BB000DF91BFC102D280F09F3740F491110EF413
:104BC00014C260E070E080E89FE3089526F01B16B1
:104BD000611D711D811D1BC135C1EFD008F481E03D
:104BE000089577D1E395B6C10CD0A3C16AD140F046
:104BF00061D130F021F45F3F19F003C15111F5C1CB
:104C000031C1B9D198F39923C9F35523B1F3951B59
:104C1000550BBB27AA2762177307840738F09F5FDD
:104C20005F4F220F331F441FAA1FA9F333D00E2E4C
:104C30003AF0E0E830D091505040E695001CCAF7B9
:104C400029D0FE2F27D0660F771F881FBB1F26177E
:104C500037074807AB07B0E809F0BB0B802DBF0151
:104C6000FF2793585F4F2AF09E3F510568F0C9C057
:104C7000BCC15F3FECF3983EDCF386957795679572
:104C8000B795F7959F5FC9F7880F911D9695879502
:104C900097F90895E1E0660F771F881FBB1F621721
:104CA00073078407BA0720F0621B730B840BBA0BDF
:104CB000EE1F88F7E095089504D06894B11195C16E
:104CC000089561D188F09F5790F0B92F9927B75177
:104CD000A0F0D1F0660F771F881F991F1AF0BA95C0
:104CE000C9F712C0B13081F07FD1B1E008957CC125
:104CF000672F782F8827B85F39F0B93FCCF38695B6
:104D000077956795B395D9F73EF490958095709512
:104D100061957F4F8F4F9F4F0895E89409C097FB8F
:104D20003EF490958095709561957F4F8F4F9F4F82
:104D30009923A9F0F92F96E9BB279395F6958795C6
:104D400077956795B795F111F8CFFAF4BB0F11F489
:104D500060FF1BC06F5F7F4F8F4F9F4F16C0882330
:104D600011F096E911C0772321F09EE8872F762F66
:104D700005C0662371F096E8862F70E060E02AF0A7
:104D80009A95660F771F881FDAF7880F9695879593
:104D900097F9089512D180F09F3740F491110EF0E9
:104DA00024C160E070E080E89FEB089526F41B16B4
:104DB000611D711D811D2BC045C0990F0008550F45
:104DC000AA0BE0E8FEEF16161706E807F907C0F091
:104DD00012161306E407F50798F0621B730B840B99
:104DE000950B39F40A2661F0232B242B252B21F473
:104DF00008950A2609F4A140A6958FEF811D811D13
:104E0000089597F99F6780E870E060E0089588232F
:104E100071F4772321F09850872B762F07C06623F3
:104E200011F499270DC09051862B70E060E02AF0B4
:104E30009A95660F771F881FDAF7880F96958795E2
:104E400097F908959F3F49F0915028F486957795FA
:104E50006795B7959F5F80389F4F880F9695879588
:104E600097F908959FEF80EC0895DF93CF931F93F8
:104E70000F93FF92EF92DF927B018C01689405C043
:104E8000DA2EEF0196D1FE01E894A5912591359196
:104E900045915591AEF3EF01D8DDFE019701A801D0
:104EA000DA9479F7DF90EF90FF900F911F91CF91F7
:104EB000DF91089500240A941616170618060906AD
:104EC000089500240A941216130614060506089580
:104ED000C9CF59D0E8F3E894EFEFBB273FE048ECA7
:104EE0005FE76B3D73078407950708F1FF279F571E
:104EF000B25A6A4D7F40894CF04032F4BE5565424B
:104F0000704F8643FF4F0894EE1F915030F0BB0F57
:104F1000661F771F881FFF1FEBCF9EE7882332F0A5
:104F2000BB0F661F771F881F9A95C1F79395E09571
:104F300089CF092E0394000C11F4882352F0BB0F83
:104F400040F4BF2B11F460FF04C06F5F7F4F8F4FA1
:104F50009F4F0895EF93E0FF06C0A2EA2AED3FE0DD
:104F600049EC5FEB72DDE5DF0F90039401FC905894
:104F7000E5E9F0E0FEC157FD9058440F551F59F088
:104F80005F3F71F04795880F97FB991F61F09F3F36
:104F900079F087950895121613061406551FF2CF5F
:104FA0004695F1DF08C0161617061806991FF1CFAF
:104FB00086957105610508940895E5DFA0F0BEE7C8
:104FC000B91788F4BB279F3860F41616B11D672FF8
:104FD000782F8827985FF7CF869577956795B11DCD
:104FE00093959639C8F30895E894BB2766277727E9
:104FF000CB0197F90895E1DE08F48FEF08955ADFA9
:1050000019F05FDF09F02ECFFCCEB901CA011ACF2B
:105010009F775F77B0DF98F39923B9F35523B9F3FE
:10502000FF27951758F4E52FE91BED3070F75E3B2D
:1050300010F0F1E41CC09034E0F40AC0E92FE51B45
:10504000ED3028F79E3B10F0F1E411C0503488F4A5
:10505000F9EA88232AF09A95660F771F881FDAF7F6
:1050600044232AF05A95220F331F441FDAF79F1B5F
:105070005F1BFF931F930F93FF92EF9279018A01B9
:10508000BB27AB2F9B01AC0196D09701A801BF9322
:105090007B018C01AA27BA2FB901CA018CD0AF912C
:1050A0009701A801EF90FF900F911F91CEDC41DF97
:1050B00001D14F9140FF0895552747FD509509C0F4
:1050C0009B01AC0160E070E080E89FE38DCD99CE5C
:1050D000B9CE59DFE8F39923D9F3940F511DBBF3EF
:1050E0009150504094F059F0882332F0660F771FAA
:1050F000881F91505040C1F79E3F510544F7880FDB
:10510000911D9695879597F908955F3FACF0983E6D
:105110009CF0BB27869577956795B79508F4B160A5
:105120009395C1F7BB0F58F711F460FFE8CF6F5F9D
:105130007F4F8F4F9F4FE3CF58CF25DF58F19E57BA
:1051400058F19851A0F0E9F0983020F5092E9927F0
:10515000660F771F881F991F0A94D1F712C0062E79
:10516000672F782F8827985F11F4000C07C0993FAC
:10517000B4F38695779567959395D9F7611D711D61
:10518000811D3EF490958095709561957F4F8F4F6E
:105190009F4F0895689429CF27CF0BD0CACE8ADEBF
:1051A00028F08FDE18F0952309F02BCE5BCE11246A
:1051B0001CCFE1DEA0F3959FD1F3950F50E0551F72
:1051C000629FF001729FBB27F00DB11D639FAA275C
:1051D000F00DB11DAA1F649F6627B00DA11D661FAB
:1051E000829F2227B00DA11D621F739FB00DA11DCC
:1051F000621F839FA00D611D221F749F3327A00D86
:10520000611D231F849F600D211D822F762F6A2F21
:1052100011249F5750408AF0E1F088234AF0EE0FA6
:10522000FF1FBB1F661F771F881F91505040A9F7B3
:105230009E3F510570F0E5CDD8CE5F3FECF3983E30
:10524000DCF3869577956795B795F795E7959F5F1A
:10525000C1F7FE2B880F911D9695879597F90895B4
:1052600092DEE0F09E37D8F09639B8F49E3848F4D4
:10527000672F782F8827985FF9CF86957795679560
:1052800093959539D0F3B62FB1706B0F711D811DB9
:1052900020F48795779567959395B9CDD3CDA5CE15
:1052A0009F9317DE0F9007FCEE5F54CE11F40EF4BF
:1052B000D9CDC8CD68DED0F39923D9F3CEF39F576B
:1052C000550B87FF4FD056959795B0E020F4660FA9
:1052D000771F881FBB1F1F930F9300249001A0010D
:1052E0008001F001A0E80E0F1F1F0A1E511D601B58
:1052F000710B8009B50B48F4600F711F801DB51F3D
:105300000E1B1F0B0A0A510907C02E0F3F1F4A1F11
:105310000E0F1F1F0A1E511D660F771F881FBB1F10
:10532000A695F795E795F8F60617170708065B07A1
:10533000211D311D411D0F911F91B901842F9158DD
:10534000880F9695879508959B01AC0126CF35DE91
:1053500020F09F3708F449CE5ACD74CD2EDD880B4E
:10536000990B089591505040660F771F881FD2F710
:1053700008959F938F937F936F93FF93EF939B0178
:10538000AC010BDFEF91FF9170DD2F913F914F91B9
:105390005F9103CF629FD001739FF001829FE00D68
:1053A000F11D649FE00DF11D929FF00D839FF00DA4
:1053B000749FF00D659FF00D9927729FB00DE11D50
:1053C000F91F639FB00DE11DF91FBD01CF0111242D
:1053D0000895A1E21A2EAA1BBB1BFD010DC0AA1F36
:1053E000BB1FEE1FFF1FA217B307E407F50720F04E
:1053F000A21BB30BE40BF50B661F771F881F991FC9
:105400001A9469F760957095809590959B01AC0111
:10541000BD01CF01089597FB092E05260ED057FD3B
:1054200004D0D7DF0AD0001C38F450954095309551
:1054300021953F4F4F4F5F4F0895F6F79095809518
:10544000709561957F4F8F4F9F4F0895911106C0C2
:10545000803219F089508550D0F708959927882710
:1054600008952F923F924F925F926F927F928F9208
:105470009F92AF92BF92CF92DF92EF92FF920F93E3
:105480001F93CF93DF93CDB7DEB7CA1BDB0B0FB6ED
:10549000F894DEBF0FBECDBF09942A8839884888AA
:1054A0005F846E847D848C849B84AA84B984C88440
:1054B000DF80EE80FD800C811B81AA81B981CE0F37
:1054C000D11D0FB6F894DEBF0FBECDBFED0108951C
:0454D000F894FFCF7E
:1054D4004D506F733A5B002C005D2C57506F733A3C
:0654E4005B005D0D0A00F3
:00000001FF
